000: 00 0c     IRQ0 Vector 000Ch
002: 00 0c     IRQ1 Vector 000Ch
004: 00 0c     IRQ2 Vector 000Ch
006: 00 0c     IRQ3 Vector 000Ch
008: 0f a4     IRQ4 Vector 0FA4h
00a: 0f b2     IRQ5 Vector 0FB2h
00c: ff        NOP  
00d: 8f        DI   
00e: 5f        Illegal
00f: 31 f0     SRP  #F0h
011: e6 02 ff  LD   P2, #FFh
014: e6 01 ff  LD   P1, #FFh
017: e6 00 ff  LD   P0, #FFh
01a: bc 20     LD   R11, #20h
01c: 1c 0c     LD   R1, #0Ch
01e: 2c 8f     LD   R2, #8Fh
020: 3c 7f     LD   R3, #7Fh
022: 4c ff     LD   R4, #FFh
024: 5c ff     LD   R5, #FFh
026: 6c 30     LD   R6, #30h
028: b0 e7     CLR  R7
02a: 8c 05     LD   R8, #05h
02c: 9c 03     LD   R9, #03h
02e: b0 ec     CLR  R12
030: b0 ee     CLR  R14
032: fc 7f     LD   R15, #7Fh
034: 31 00     SRP  #00h
036: b0 03     CLR  P3
038: 4c 06     LD   R4, #06h
03a: 5c 01     LD   R5, #01h
03c: 5f        Illegal
03d: f3 45     LD   @R4, R5
03f: a3 54     CP   R5, @R4
041: ed 00 c2  JP   NZ, 00C2h
044: 90 e5     RL   R5
046: fb f5     JR   NC, 003Dh
048: b1 e4     CLR  @R4
04a: 4e        INC  R4
04b: db ed     JR   PL, 003Ah
04d: 31 10     SRP  #10h
04f: d6 0f de  CALL 0FDEh
052: 7b 6e     JR   C, 00C2h
054: e6 0a 44  LD   0Ah, #44h
057: d6 0d 3d  CALL 0D3Dh
05a: 76 03 01  TM   P3, #01h
05d: eb 05     JR   NZ, 0064h
05f: e6 09 03  LD   09h, #03h
062: 8b 05     JR   0069h
064: b0 08     CLR  08h
066: e6 09 02  LD   09h, #02h
069: e6 02 ff  LD   P2, #FFh
06c: e6 03 ff  LD   P3, #FFh
06f: e6 1f 40  LD   1Fh, #40h
072: d6 06 67  CALL 0667h
075: 2c aa     LD   R2, #AAh
077: d6 07 8a  CALL 078Ah
07a: 31 10     SRP  #10h
07c: 9f        EI   
07d: e6 0d 55  LD   0Dh, #55h
080: 5f        Illegal
081: e6 68 20  LD   68h, #20h
084: 46 fb a0  OR   IMR, #A0h
087: 46 f1 08  OR   TMR, #08h
08a: d6 02 75  CALL 0275h
08d: d6 00 d0  CALL 00D0h
090: d6 01 c8  CALL 01C8h
093: d6 00 b2  CALL 00B2h
096: 7d 0b 11  JP   C, 0B11h
099: 9f        EI   
09a: d6 02 75  CALL 0275h
09d: d6 0e 66  CALL 0E66h
0a0: d6 00 b2  CALL 00B2h
0a3: 7d 0b 11  JP   C, 0B11h
0a6: 9f        EI   
0a7: d6 0e 66  CALL 0E66h
0aa: d6 00 b2  CALL 00B2h
0ad: 7d 0b 11  JP   C, 0B11h
0b0: 8b c8     JR   007Ah
0b2: 76 02 40  TM   P2, #40h
0b5: ed 00 c0  JP   NZ, 00C0h
0b8: 76 02 80  TM   P2, #80h
0bb: 6b 03     JR   Z, 00C0h
0bd: 8f        DI   
0be: df        SCF  
0bf: af        RET  
0c0: cf        RCF  
0c1: af        RET  
0c2: e6 0a 44  LD   0Ah, #44h
0c5: e6 02 ff  LD   P2, #FFh
0c8: 2c fc     LD   R2, #FCh
0ca: d6 07 8a  CALL 078Ah
0cd: 8d 0b 11  JP   0B11h
0d0: 31 10     SRP  #10h
0d2: e6 0d 55  LD   0Dh, #55h
0d5: e6 68 20  LD   68h, #20h
0d8: 5f        Illegal
0d9: e6 02 ff  LD   P2, #FFh
0dc: e6 00 ff  LD   P0, #FFh
0df: e6 f8 05  LD   P01M, #05h
0e2: e6 f6 30  LD   P2M, #30h
0e5: e6 f7 00  LD   P3M, #00h
0e8: b0 13     CLR  13h
0ea: 4c 08     LD   R4, #08h
0ec: e6 04 7f  LD   04h, #7Fh
0ef: e4 04 01  LD   P1, 04h
0f2: d6 01 35  CALL 0135h
0f5: 7b 38     JR   C, 012Fh
0f7: 20 13     INC  13h
0f9: df        SCF  
0fa: c0 04     RRC  04h
0fc: 4a f1     DJNZ R4, 00EFh
0fe: e6 01 ff  LD   P1, #FFh
101: 4c 04     LD   R4, #04h
103: e6 04 ef  LD   04h, #EFh
106: e4 04 00  LD   P0, 04h
109: d6 01 35  CALL 0135h
10c: 7b 21     JR   C, 012Fh
10e: 20 13     INC  13h
110: df        SCF  
111: 10 04     RLC  04h
113: 4a f1     DJNZ R4, 0106h
115: e6 00 ff  LD   P0, #FFh
118: 4c 04     LD   R4, #04h
11a: e6 04 fe  LD   04h, #FEh
11d: e4 04 02  LD   P2, 04h
120: d6 01 35  CALL 0135h
123: 7b 0a     JR   C, 012Fh
125: 20 13     INC  13h
127: 46 04 f0  OR   04h, #F0h
12a: df        SCF  
12b: 10 04     RLC  04h
12d: 4a ee     DJNZ R4, 011Dh
12f: e6 02 ff  LD   P2, #FFh
132: 9f        EI   
133: af        RET  
134: bf        IRET 
135: 7c 02     LD   R7, #02h
137: 7a fe     DJNZ R7, 0137h
139: 76 02 40  TM   P2, #40h
13c: eb 05     JR   NZ, 0143h
13e: 76 02 80  TM   P2, #80h
141: eb 2d     JR   NZ, 0170h
143: b0 ed     CLR  R13
145: e6 05 08  LD   05h, #08h
148: 7c 0f     LD   R7, #0Fh
14a: 54 00 e7  AND  R7, P0
14d: 76 03 08  TM   P3, #08h
150: eb 21     JR   NZ, 0173h
152: 76 03 02  TM   P3, #02h
155: eb 21     JR   NZ, 0178h
157: 5c 30     LD   R5, #30h
159: 54 02 e5  AND  R5, P2
15c: 90 e5     RL   R5
15e: 42 75     OR   R7, R5
160: 60 e7     COM  R7
162: 6b 0b     JR   Z, 016Fh
164: cf        RCF  
165: c0 e7     RRC  R7
167: 7b 14     JR   C, 017Dh
169: de        INC  R13
16a: 00 05     DEC  05h
16c: eb f6     JR   NZ, 0164h
16e: cf        RCF  
16f: af        RET  
170: 8f        DI   
171: df        SCF  
172: af        RET  
173: 46 e7 10  OR   R7, #10h
176: 8b da     JR   0152h
178: 46 e7 80  OR   R7, #80h
17b: 8b da     JR   0157h
17d: 58 13     LD   R5, 13h
17f: 90 e5     RL   R5
181: 90 e5     RL   R5
183: 90 e5     RL   R5
185: 56 e5 f8  AND  R5, #F8h
188: 42 5d     OR   R5, R13
18a: eb 02     JR   NZ, 018Eh
18c: 5c 80     LD   R5, #80h
18e: 6c 56     LD   R6, #56h
190: e3 a6     LD   R10, @R6
192: cf        RCF  
193: 90 ea     RL   R10
195: 7b 09     JR   C, 01A0h
197: 6e        INC  R6
198: 6e        INC  R6
199: a6 e6 66  CP   R6, #66h
19c: 1b f2     JR   LT, 0190h
19e: 8b 0e     JR   01AEh
1a0: 6e        INC  R6
1a1: e3 a6     LD   R10, @R6
1a3: a2 a5     CP   R10, R5
1a5: eb f1     JR   NZ, 0198h
1a7: 00 e6     DEC  R6
1a9: 47 e6 10  OR   @R6, #10h
1ac: 8b bb     JR   0169h
1ae: 6c 56     LD   R6, #56h
1b0: e3 a6     LD   R10, @R6
1b2: cf        RCF  
1b3: 90 ea     RL   R10
1b5: 7b 08     JR   C, 01BFh
1b7: 47 e6 90  OR   @R6, #90h
1ba: 6e        INC  R6
1bb: f3 65     LD   @R6, R5
1bd: 8b aa     JR   0169h
1bf: 6e        INC  R6
1c0: 6e        INC  R6
1c1: a6 e6 66  CP   R6, #66h
1c4: eb ea     JR   NZ, 01B0h
1c6: 8b a1     JR   0169h
1c8: 4c 56     LD   R4, #56h
1ca: e3 64     LD   R6, @R4
1cc: 76 e6 80  TM   R6, #80h
1cf: eb 02     JR   NZ, 01D3h
1d1: 8b 4a     JR   021Dh
1d3: 76 e6 10  TM   R6, #10h
1d6: eb 0c     JR   NZ, 01E4h
1d8: 76 e6 20  TM   R6, #20h
1db: eb 20     JR   NZ, 01FDh
1dd: b1 e4     CLR  @R4
1df: 4e        INC  R4
1e0: b1 e4     CLR  @R4
1e2: 8b 3a     JR   021Eh
1e4: 57 e4 ef  AND  @R4, #EFh
1e7: 76 e6 20  TM   R6, #20h
1ea: eb 27     JR   NZ, 0213h
1ec: 56 e6 05  AND  R6, #05h
1ef: a6 e6 05  CP   R6, #05h
1f2: eb 05     JR   NZ, 01F9h
1f4: 47 e4 27  OR   @R4, #27h
1f7: 8b 24     JR   021Dh
1f9: 21 e4     INC  @R4
1fb: 8b 20     JR   021Dh
1fd: 56 e6 07  AND  R6, #07h
200: eb 16     JR   NZ, 0218h
202: 77 e4 08  TM   @R4, #08h
205: eb 07     JR   NZ, 020Eh
207: b1 e4     CLR  @R4
209: 4e        INC  R4
20a: b1 e4     CLR  @R4
20c: 8b 10     JR   021Eh
20e: 47 e4 40  OR   @R4, #40h
211: 8b 0a     JR   021Dh
213: 47 e4 07  OR   @R4, #07h
216: 8b 05     JR   021Dh
218: 01 e4     DEC  @R4
21a: 47 e4 80  OR   @R4, #80h
21d: 4e        INC  R4
21e: 4e        INC  R4
21f: a6 e4 66  CP   R4, #66h
222: 1b a6     JR   LT, 01CAh
224: af        RET  
225: a6 ec 43  CP   R12, #43h
228: eb 03     JR   NZ, 022Dh
22a: ec 01     LD   R14, #01h
22c: af        RET  
22d: a6 ec 4e  CP   R12, #4Eh
230: eb 03     JR   NZ, 0235h
232: ec 02     LD   R14, #02h
234: af        RET  
235: a6 ec 36  CP   R12, #36h
238: eb 03     JR   NZ, 023Dh
23a: ec 10     LD   R14, #10h
23c: af        RET  
23d: 1c 71     LD   R1, #71h
23f: 0c 02     LD   R0, #02h
241: c2 20     LDC  R2, @RR0
243: a2 c2     CP   R12, R2
245: 6b 19     JR   Z, 0260h
247: 1e        INC  R1
248: a6 e2 00  CP   R2, #00h
24b: eb f4     JR   NZ, 0241h
24d: 1c 66     LD   R1, #66h
24f: 0c 02     LD   R0, #02h
251: c2 20     LDC  R2, @RR0
253: a2 c2     CP   R12, R2
255: 6b 0c     JR   Z, 0263h
257: 1e        INC  R1
258: a6 e2 00  CP   R2, #00h
25b: eb f4     JR   NZ, 0251h
25d: b0 ee     CLR  R14
25f: af        RET  
260: ec 08     LD   R14, #08h
262: af        RET  
263: ec 04     LD   R14, #04h
265: af        RET  
266: 32 4a     SBC  R4, R10
268: 52 2a     AND  R2, R10
26a: 4b 53     JR   OV, 02BFh
26c: 48 4f     LD   R4, 4Fh
26e: 2f        Illegal
26f: 37 00 5e  SBC  @00h, #5Eh
272: 47 4d 00  OR   @4Dh, #00h
275: 5f        Illegal
276: e6 0d 55  LD   0Dh, #55h
279: e6 68 20  LD   68h, #20h
27c: 4c 44     LD   R4, #44h
27e: e3 64     LD   R6, @R4
280: a6 e6 00  CP   R6, #00h
283: 6b 30     JR   Z, 02B5h
285: d6 0e e5  CALL 0EE5h
288: 7b 2b     JR   C, 02B5h
28a: 48 0a     LD   R4, 0Ah
28c: 00 e4     DEC  R4
28e: 49 0a     LD   0Ah, R4
290: 5c 11     LD   R5, #11h
292: 4c 45     LD   R4, #45h
294: e3 24     LD   R2, @R4
296: 00 e4     DEC  R4
298: f3 42     LD   @R4, R2
29a: 4e        INC  R4
29b: 4e        INC  R4
29c: 00 e5     DEC  R5
29e: eb f4     JR   NZ, 0294h
2a0: b0 55     CLR  55h
2a2: 56 1f 7f  AND  1Fh, #7Fh
2a5: 5f        Illegal
2a6: 5c 05     LD   R5, #05h
2a8: 6c 50     LD   R6, #50h
2aa: 76 02 40  TM   P2, #40h
2ad: 6b 04     JR   Z, 02B3h
2af: 6a f9     DJNZ R6, 02AAh
2b1: 5a f5     DJNZ R5, 02A8h
2b3: 8b c0     JR   0275h
2b5: 9f        EI   
2b6: 5f        Illegal
2b7: 4c 56     LD   R4, #56h
2b9: e3 64     LD   R6, @R4
2bb: 76 e6 80  TM   R6, #80h
2be: eb 0a     JR   NZ, 02CAh
2c0: 9f        EI   
2c1: 5f        Illegal
2c2: 4e        INC  R4
2c3: 4e        INC  R4
2c4: a6 e4 66  CP   R4, #66h
2c7: eb f0     JR   NZ, 02B9h
2c9: af        RET  
2ca: e4 0a 69  LD   69h, 0Ah
2cd: 76 e6 20  TM   R6, #20h
2d0: eb 02     JR   NZ, 02D4h
2d2: 8b ec     JR   02C0h
2d4: 76 e6 08  TM   R6, #08h
2d7: eb 64     JR   NZ, 033Dh
2d9: d6 06 a6  CALL 06A6h
2dc: 7b e2     JR   C, 02C0h
2de: 4e        INC  R4
2df: 70 e4     PUSH R4
2e1: e3 c4     LD   R12, @R4
2e3: a6 09 03  CP   09h, #03h
2e6: 6b 2d     JR   Z, 0315h
2e8: d6 02 25  CALL 0225h
2eb: d6 03 90  CALL 0390h
2ee: 50 e4     POP  R4
2f0: 76 1f 80  TM   1Fh, #80h
2f3: eb 25     JR   NZ, 031Ah
2f5: a6 09 03  CP   09h, #03h
2f8: eb 0f     JR   NZ, 0309h
2fa: 28 ec     LD   R2, R12
2fc: d6 0e 26  CALL 0E26h
2ff: 76 05 01  TM   05h, #01h
302: eb 05     JR   NZ, 0309h
304: e6 0c 00  LD   0Ch, #00h
307: 8b 05     JR   030Eh
309: e4 06 0c  LD   0Ch, 06h
30c: c9 0b     LD   0Bh, R12
30e: 00 e4     DEC  R4
310: 47 e4 08  OR   @R4, #08h
313: 8b ab     JR   02C0h
315: d6 0e 10  CALL 0E10h
318: 8b d4     JR   02EEh
31a: e4 69 0a  LD   0Ah, 69h
31d: a6 69 55  CP   69h, #55h
320: 9b 1a     JR   GE, 033Ch
322: 00 69     DEC  69h
324: a7 69 ff  CP   @69h, #FFh
327: 6b 05     JR   Z, 032Eh
329: 20 69     INC  69h
32b: e7 69 ff  LD   @69h, #FFh
32e: 20 69     INC  69h
330: e4 69 0a  LD   0Ah, 69h
333: b1 69     CLR  @69h
335: 20 69     INC  69h
337: a6 69 55  CP   69h, #55h
33a: 1b f7     JR   LT, 0333h
33c: af        RET  
33d: 76 e6 40  TM   R6, #40h
340: eb 03     JR   NZ, 0345h
342: 8d 02 c0  JP   02C0h
345: 4e        INC  R4
346: e3 c4     LD   R12, @R4
348: a6 09 03  CP   09h, #03h
34b: 6b 37     JR   Z, 0384h
34d: 70 e4     PUSH R4
34f: d6 02 25  CALL 0225h
352: d6 04 d4  CALL 04D4h
355: 50 e4     POP  R4
357: 76 1f 80  TM   1Fh, #80h
35a: eb be     JR   NZ, 031Ah
35c: a5 e4 0b  CP   0Bh, @R4
35f: eb 0b     JR   NZ, 036Ch
361: b0 0b     CLR  0Bh
363: b1 e4     CLR  @R4
365: 00 e4     DEC  R4
367: b1 e4     CLR  @R4
369: 8d 02 c0  JP   02C0h
36c: a7 e4 43  CP   @R4, #43h
36f: eb 0c     JR   NZ, 037Dh
371: a6 0b 81  CP   0Bh, #81h
374: 6b eb     JR   Z, 0361h
376: a6 0b 82  CP   0Bh, #82h
379: eb e8     JR   NZ, 0363h
37b: 8b e4     JR   0361h
37d: a6 0b 82  CP   0Bh, #82h
380: eb e1     JR   NZ, 0363h
382: 8b dd     JR   0361h
384: a6 0b 82  CP   0Bh, #82h
387: eb 02     JR   NZ, 038Bh
389: b0 0b     CLR  0Bh
38b: d6 0d ee  CALL 0DEEh
38e: 8b c7     JR   0357h
390: 76 ee 04  TM   R14, #04h
393: ed 04 36  JP   NZ, 0436h
396: 76 18 40  TM   18h, #40h
399: ed 04 c5  JP   NZ, 04C5h
39c: 76 ee 02  TM   R14, #02h
39f: ed 04 22  JP   NZ, 0422h
3a2: 76 ee 01  TM   R14, #01h
3a5: eb 2d     JR   NZ, 03D4h
3a7: 76 ee 08  TM   R14, #08h
3aa: eb 5e     JR   NZ, 040Ah
3ac: 76 ee 10  TM   R14, #10h
3af: ed 04 a7  JP   NZ, 04A7h
3b2: 76 e9 02  TM   R9, #02h
3b5: 6b 06     JR   Z, 03BDh
3b7: d6 04 17  CALL 0417h
3ba: 46 e9 10  OR   R9, #10h
3bd: a6 08 00  CP   08h, #00h
3c0: eb 0a     JR   NZ, 03CCh
3c2: d6 0f d3  CALL 0FD3h
3c5: d6 07 8a  CALL 078Ah
3c8: d6 06 1f  CALL 061Fh
3cb: af        RET  
3cc: d6 0f ca  CALL 0FCAh
3cf: 56 e2 7f  AND  R2, #7Fh
3d2: 8b f1     JR   03C5h
3d4: 76 e9 01  TM   R9, #01h
3d7: ed 04 bd  JP   NZ, 04BDh
3da: 76 18 08  TM   18h, #08h
3dd: ed 04 bd  JP   NZ, 04BDh
3e0: 76 e9 20  TM   R9, #20h
3e3: ed 04 bd  JP   NZ, 04BDh
3e6: 46 e9 02  OR   R9, #02h
3e9: 76 18 7d  TM   18h, #7Dh
3ec: eb 08     JR   NZ, 03F6h
3ee: 1c 83     LD   R1, #83h
3f0: 0c 08     LD   R0, #08h
3f2: d6 06 0e  CALL 060Eh
3f5: af        RET  
3f6: 76 18 05  TM   18h, #05h
3f9: 6b 03     JR   Z, 03FEh
3fb: 46 67 02  OR   67h, #02h
3fe: 76 18 30  TM   18h, #30h
401: 6d 04 86  JP   Z, 0486h
404: 46 e9 08  OR   R9, #08h
407: 8d 04 86  JP   0486h
40a: 76 e9 02  TM   R9, #02h
40d: 6b 6f     JR   Z, 047Eh
40f: d6 04 17  CALL 0417h
412: 46 e9 10  OR   R9, #10h
415: 8b 67     JR   047Eh
417: 56 e9 fd  AND  R9, #FDh
41a: 0c 08     LD   R0, #08h
41c: 1c 9b     LD   R1, #9Bh
41e: d6 06 0e  CALL 060Eh
421: af        RET  
422: 76 e9 02  TM   R9, #02h
425: 6b 03     JR   Z, 042Ah
427: d6 04 17  CALL 0417h
42a: 76 18 30  TM   18h, #30h
42d: ed 04 b6  JP   NZ, 04B6h
430: 1c 8c     LD   R1, #8Ch
432: 0c 08     LD   R0, #08h
434: 8b bc     JR   03F2h
436: 76 e9 02  TM   R9, #02h
439: 6b 03     JR   Z, 043Eh
43b: d6 04 17  CALL 0417h
43e: 28 18     LD   R2, 18h
440: 56 e2 07  AND  R2, #07h
443: 6b 39     JR   Z, 047Eh
445: 76 18 02  TM   18h, #02h
448: eb 46     JR   NZ, 0490h
44a: 76 18 01  TM   18h, #01h
44d: eb 1f     JR   NZ, 046Eh
44f: 76 e9 80  TM   R9, #80h
452: 6b 15     JR   Z, 0469h
454: 0c 08     LD   R0, #08h
456: 1c a3     LD   R1, #A3h
458: d6 06 0e  CALL 060Eh
45b: 1c 9f     LD   R1, #9Fh
45d: 0c 08     LD   R0, #08h
45f: d6 06 0e  CALL 060Eh
462: 8b 1a     JR   047Eh
464: 46 e9 40  OR   R9, #40h
467: 8b 0d     JR   0476h
469: 46 e9 80  OR   R9, #80h
46c: 8b ed     JR   045Bh
46e: 76 e9 40  TM   R9, #40h
471: 6b f1     JR   Z, 0464h
473: d6 05 43  CALL 0543h
476: d6 04 1a  CALL 041Ah
479: 76 18 04  TM   18h, #04h
47c: eb dd     JR   NZ, 045Bh
47e: 2c e0     LD   R2, #E0h
480: d6 07 8a  CALL 078Ah
483: 8d 03 bd  JP   03BDh
486: 56 e9 fd  AND  R9, #FDh
489: 8b f3     JR   047Eh
48b: 46 67 01  OR   67h, #01h
48e: 8b ee     JR   047Eh
490: 76 18 40  TM   18h, #40h
493: eb 0d     JR   NZ, 04A2h
495: 76 18 05  TM   18h, #05h
498: eb f1     JR   NZ, 048Bh
49a: 46 18 40  OR   18h, #40h
49d: d6 05 43  CALL 0543h
4a0: 8b dc     JR   047Eh
4a2: d6 04 1a  CALL 041Ah
4a5: 8b f3     JR   049Ah
4a7: 76 e9 02  TM   R9, #02h
4aa: 6b 03     JR   Z, 04AFh
4ac: d6 04 17  CALL 0417h
4af: 76 18 65  TM   18h, #65h
4b2: 6b ca     JR   Z, 047Eh
4b4: 8b 94     JR   044Ah
4b6: 1c 95     LD   R1, #95h
4b8: 0c 08     LD   R0, #08h
4ba: 8d 03 f2  JP   03F2h
4bd: 46 e9 01  OR   R9, #01h
4c0: cc 81     LD   R12, #81h
4c2: 8d 03 bd  JP   03BDh
4c5: d6 04 1a  CALL 041Ah
4c8: 76 1f 80  TM   1Fh, #80h
4cb: ed 04 d1  JP   NZ, 04D1h
4ce: 56 18 bf  AND  18h, #BFh
4d1: 8d 03 9c  JP   039Ch
4d4: 76 ee 01  TM   R14, #01h
4d7: ed 05 ac  JP   NZ, 05ACh
4da: 76 ee 02  TM   R14, #02h
4dd: 6b 01     JR   Z, 04E0h
4df: af        RET  
4e0: a6 ee 00  CP   R14, #00h
4e3: ed 06 06  JP   NZ, 0606h
4e6: 56 e9 ef  AND  R9, #EFh
4e9: a6 08 00  CP   08h, #00h
4ec: 6b 08     JR   Z, 04F6h
4ee: d6 0f ca  CALL 0FCAh
4f1: 46 e2 80  OR   R2, #80h
4f4: 8b 08     JR   04FEh
4f6: 2c f0     LD   R2, #F0h
4f8: d6 07 8a  CALL 078Ah
4fb: d6 0f d3  CALL 0FD3h
4fe: d6 07 8a  CALL 078Ah
501: a6 ec 3e  CP   R12, #3Eh
504: 6d 05 86  JP   Z, 0586h
507: a6 ec 39  CP   R12, #39h
50a: 6b 6b     JR   Z, 0577h
50c: a6 ec 47  CP   R12, #47h
50f: 6d 05 fa  JP   Z, 05FAh
512: a6 ec 40  CP   R12, #40h
515: 6d 05 f3  JP   Z, 05F3h
518: a6 ec 5a  CP   R12, #5Ah
51b: 6d 05 fe  JP   Z, 05FEh
51e: a6 ec 5e  CP   R12, #5Eh
521: 6d 06 02  JP   Z, 0602h
524: 76 ee 04  TM   R14, #04h
527: 6b 40     JR   Z, 0569h
529: a4 0b ec  CP   R12, 0Bh
52c: eb 48     JR   NZ, 0576h
52e: 56 e9 3f  AND  R9, #3Fh
531: 56 67 fc  AND  67h, #FCh
534: 76 18 07  TM   18h, #07h
537: 6b 3d     JR   Z, 0576h
539: 76 18 02  TM   18h, #02h
53c: eb 1a     JR   NZ, 0558h
53e: 76 18 04  TM   18h, #04h
541: eb 08     JR   NZ, 054Bh
543: 1c a6     LD   R1, #A6h
545: 0c 08     LD   R0, #08h
547: d6 06 0e  CALL 060Eh
54a: af        RET  
54b: 1c a3     LD   R1, #A3h
54d: 0c 08     LD   R0, #08h
54f: d6 06 0e  CALL 060Eh
552: 76 18 01  TM   18h, #01h
555: eb ec     JR   NZ, 0543h
557: af        RET  
558: 76 18 05  TM   18h, #05h
55b: eb 19     JR   NZ, 0576h
55d: d6 04 1a  CALL 041Ah
560: 76 1f 80  TM   1Fh, #80h
563: eb 03     JR   NZ, 0568h
565: 56 18 bf  AND  18h, #BFh
568: af        RET  
569: 76 ee 10  TM   R14, #10h
56c: 6b 08     JR   Z, 0576h
56e: 56 e9 3f  AND  R9, #3Fh
571: 76 18 05  TM   18h, #05h
574: eb c8     JR   NZ, 053Eh
576: af        RET  
577: d6 05 95  CALL 0595h
57a: 56 e9 bf  AND  R9, #BFh
57d: 56 18 fe  AND  18h, #FEh
580: 76 18 02  TM   18h, #02h
583: eb 0c     JR   NZ, 0591h
585: af        RET  
586: d6 05 95  CALL 0595h
589: 56 e9 7f  AND  R9, #7Fh
58c: 56 18 fb  AND  18h, #FBh
58f: 8b ef     JR   0580h
591: 46 18 80  OR   18h, #80h
594: af        RET  
595: 76 67 01  TM   67h, #01h
598: 6b 07     JR   Z, 05A1h
59a: d6 05 43  CALL 0543h
59d: 56 67 3f  AND  67h, #3Fh
5a0: af        RET  
5a1: 76 67 02  TM   67h, #02h
5a4: eb 01     JR   NZ, 05A7h
5a6: af        RET  
5a7: 46 e9 02  OR   R9, #02h
5aa: 8b ee     JR   059Ah
5ac: 76 e9 08  TM   R9, #08h
5af: eb 1f     JR   NZ, 05D0h
5b1: 76 e9 02  TM   R9, #02h
5b4: eb 12     JR   NZ, 05C8h
5b6: 76 e9 01  TM   R9, #01h
5b9: eb 30     JR   NZ, 05EBh
5bb: 76 e9 10  TM   R9, #10h
5be: eb 08     JR   NZ, 05C8h
5c0: 76 18 08  TM   18h, #08h
5c3: eb 26     JR   NZ, 05EBh
5c5: 56 67 fc  AND  67h, #FCh
5c8: 56 e9 ef  AND  R9, #EFh
5cb: 76 18 7d  TM   18h, #7Dh
5ce: eb 36     JR   NZ, 0606h
5d0: 1c 88     LD   R1, #88h
5d2: 0c 08     LD   R0, #08h
5d4: d6 06 0e  CALL 060Eh
5d7: 76 e9 08  TM   R9, #08h
5da: eb 0b     JR   NZ, 05E7h
5dc: 76 e9 02  TM   R9, #02h
5df: 6b 18     JR   Z, 05F9h
5e1: 56 e9 fd  AND  R9, #FDh
5e4: 8d 04 1a  JP   041Ah
5e7: 56 e9 f7  AND  R9, #F7h
5ea: af        RET  
5eb: 56 e9 fe  AND  R9, #FEh
5ee: cc 81     LD   R12, #81h
5f0: 8d 04 e9  JP   04E9h
5f3: 56 e9 ef  AND  R9, #EFh
5f6: 56 18 77  AND  18h, #77h
5f9: af        RET  
5fa: 56 e9 cf  AND  R9, #CFh
5fd: af        RET  
5fe: 56 18 6f  AND  18h, #6Fh
601: af        RET  
602: 56 18 5f  AND  18h, #5Fh
605: af        RET  
606: 2c e0     LD   R2, #E0h
608: d6 07 8a  CALL 078Ah
60b: 8d 04 e9  JP   04E9h
60e: 04 08 e1  ADD  R1, 08h
611: c2 20     LDC  R2, @RR0
613: a6 e2 00  CP   R2, #00h
616: 6b 06     JR   Z, 061Eh
618: d6 07 8a  CALL 078Ah
61b: 1e        INC  R1
61c: 8b f3     JR   0611h
61e: af        RET  
61f: a6 ec 3e  CP   R12, #3Eh
622: 6b 27     JR   Z, 064Bh
624: a6 ec 39  CP   R12, #39h
627: 6b 26     JR   Z, 064Fh
629: a6 ec 47  CP   R12, #47h
62c: 6b 2d     JR   Z, 065Bh
62e: a6 ec 40  CP   R12, #40h
631: 6b 24     JR   Z, 0657h
633: a6 ec 5a  CP   R12, #5Ah
636: 6b 27     JR   Z, 065Fh
638: a6 ec 5e  CP   R12, #5Eh
63b: 6b 26     JR   Z, 0663h
63d: a6 ec 2e  CP   R12, #2Eh
640: eb 08     JR   NZ, 064Ah
642: 76 18 02  TM   18h, #02h
645: eb 0c     JR   NZ, 0653h
647: 46 18 02  OR   18h, #02h
64a: af        RET  
64b: 46 18 04  OR   18h, #04h
64e: af        RET  
64f: 46 18 01  OR   18h, #01h
652: af        RET  
653: 56 18 fd  AND  18h, #FDh
656: af        RET  
657: 46 18 08  OR   18h, #08h
65a: af        RET  
65b: 46 e9 20  OR   R9, #20h
65e: af        RET  
65f: 46 18 10  OR   18h, #10h
662: af        RET  
663: 46 18 20  OR   18h, #20h
666: af        RET  
667: e6 06 7f  LD   06h, #7Fh
66a: e6 07 18  LD   07h, #18h
66d: b0 e4     CLR  R4
66f: bc 20     LD   R11, #20h
671: 1c 84     LD   R1, #84h
673: 0c 06     LD   R0, #06h
675: 02 14     ADD  R1, R4
677: c2 20     LDC  R2, @RR0
679: 02 b4     ADD  R11, R4
67b: f3 b2     LD   @R11, R2
67d: 4e        INC  R4
67e: a6 e4 22  CP   R4, #22h
681: eb ec     JR   NZ, 066Fh
683: af        RET  
684: ff        NOP  
685: ff        NOP  
686: ff        NOP  
687: ff        NOP  
688: ff        NOP  
689: ff        NOP  
68a: ff        NOP  
68b: bd fe ff  JP   UGT, FEFFh
68e: ff        NOP  
68f: fb ff     JR   NC, 0690h
691: ff        NOP  
692: fd ff ff  JP   NC, FFFFh
695: ff        NOP  
696: 78 ff     LD   R7, SPL
698: f2        Illegal
699: fe        INC  R15
69a: 84        Illegal
69b: 80 bd     DECW BDh
69d: 66 93 00  TCM  93h, #00h
6a0: bb ff     JR   UGT, 06A1h
6a2: f8 f9     LD   R15, IPR
6a4: 7e        INC  R7
6a5: fd 5f 70  JP   NC, 5F70h
6a8: e6 70 e4  LD   70h, #E4h
6ab: 4e        INC  R4
6ac: e3 24     LD   R2, @R4
6ae: d6 06 f8  CALL 06F8h
6b1: 7b 07     JR   C, 06BAh
6b3: d6 07 1b  CALL 071Bh
6b6: 7b 10     JR   C, 06C8h
6b8: 8b 15     JR   06CFh
6ba: d6 07 1b  CALL 071Bh
6bd: 7b 32     JR   C, 06F1h
6bf: 28 e6     LD   R2, R6
6c1: d6 06 f8  CALL 06F8h
6c4: 7b 2b     JR   C, 06F1h
6c6: 8b 07     JR   06CFh
6c8: 28 e5     LD   R2, R5
6ca: d6 07 1b  CALL 071Bh
6cd: 7b 22     JR   C, 06F1h
6cf: a6 0b 82  CP   0Bh, #82h
6d2: 6b 0f     JR   Z, 06E3h
6d4: a6 0c 00  CP   0Ch, #00h
6d7: eb 08     JR   NZ, 06E1h
6d9: e6 0c bf  LD   0Ch, #BFh
6dc: e6 0b 82  LD   0Bh, #82h
6df: 8b 02     JR   06E3h
6e1: b0 0b     CLR  0Bh
6e3: 50 e4     POP  R4
6e5: 50 e6     POP  R6
6e7: e7 e4 a0  LD   @R4, #A0h
6ea: 8b 3e     JR   072Ah
6ec: e6 0b 82  LD   0Bh, #82h
6ef: 8b f2     JR   06E3h
6f1: 9f        EI   
6f2: 50 e4     POP  R4
6f4: 50 e6     POP  R6
6f6: cf        RCF  
6f7: af        RET  
6f8: 9f        EI   
6f9: 4c 56     LD   R4, #56h
6fb: 77 e4 80  TM   @R4, #80h
6fe: eb 09     JR   NZ, 0709h
700: 4e        INC  R4
701: 4e        INC  R4
702: a6 e4 66  CP   R4, #66h
705: 1b f4     JR   LT, 06FBh
707: df        SCF  
708: af        RET  
709: 4e        INC  R4
70a: e5 e4 05  LD   05h, @R4
70d: b4 e2 05  XOR  05h, R2
710: 6b ef     JR   Z, 0701h
712: 56 05 f8  AND  05h, #F8h
715: eb ea     JR   NZ, 0701h
717: e3 54     LD   R5, @R4
719: cf        RCF  
71a: af        RET  
71b: 9f        EI   
71c: 4c 56     LD   R4, #56h
71e: 77 e4 80  TM   @R4, #80h
721: eb 0a     JR   NZ, 072Dh
723: 4e        INC  R4
724: 4e        INC  R4
725: a6 e4 66  CP   R4, #66h
728: 1b f4     JR   LT, 071Eh
72a: 8f        DI   
72b: df        SCF  
72c: af        RET  
72d: 4e        INC  R4
72e: e5 e4 05  LD   05h, @R4
731: b4 e2 05  XOR  05h, R2
734: 6b ee     JR   Z, 0724h
736: 56 05 07  AND  05h, #07h
739: eb e9     JR   NZ, 0724h
73b: e3 64     LD   R6, @R4
73d: cf        RCF  
73e: af        RET  
73f: 68 e2     LD   R6, R2
741: a8 e2     LD   R10, R2
743: 56 e6 1f  AND  R6, #1Fh
746: 1c 6a     LD   R1, #6Ah
748: 0c 07     LD   R0, #07h
74a: 02 16     ADD  R1, R6
74c: c2 20     LDC  R2, @RR0
74e: 29 07     LD   07h, R2
750: 68 ea     LD   R6, R10
752: 90 e6     RL   R6
754: 90 e6     RL   R6
756: 90 e6     RL   R6
758: 56 e6 03  AND  R6, #03h
75b: 1c 66     LD   R1, #66h
75d: 0c 07     LD   R0, #07h
75f: 02 16     ADD  R1, R6
761: c2 20     LDC  R2, @RR0
763: 29 06     LD   06h, R2
765: af        RET  
766: 40 7f     DA   7Fh
768: bf        IRET 
769: ff        NOP  
76a: 08 0a     LD   R0, 0Ah
76c: 0b 0c     JR   F, 077Ah
76e: 0d 0e 0f  JP   F, 0E0Fh
771: 10 11     RLC  11h
773: 13 16     ADC  R1, @R6
775: 18 1a     LD   R1, 1Ah
777: 1c 1e     LD   R1, #1Eh
779: 20 22     INC  22h
77b: 26 2b 2f  SUB  2Bh, #2Fh
77e: 33 37     SBC  R3, @R7
780: 3b 40     JR   ULE, 07C2h
782: 45 4d 55  OR   55h, @4Dh
785: 5e        INC  R5
786: 66 6f 79  TCM  6Fh, #79h
789: 7f        Illegal
78a: 76 1f 80  TM   1Fh, #80h
78d: 6b 01     JR   Z, 0790h
78f: af        RET  
790: a6 0a 54  CP   0Ah, #54h
793: eb 04     JR   NZ, 0799h
795: 46 1f 80  OR   1Fh, #80h
798: af        RET  
799: f5 e2 0a  LD   @R2, 0Ah
79c: 20 0a     INC  0Ah
79e: af        RET  
79f: 8f        DI   
7a0: d6 07 b4  CALL 07B4h
7a3: a4 43 15  CP   15h, 43h
7a6: ed 00 0d  JP   NZ, 000Dh
7a9: 9f        EI   
7aa: af        RET  
7ab: 8f        DI   
7ac: d6 07 b4  CALL 07B4h
7af: e4 15 43  LD   43h, 15h
7b2: 9f        EI   
7b3: af        RET  
7b4: 31 00     SRP  #00h
7b6: b0 15     CLR  15h
7b8: 4c 06     LD   R4, #06h
7ba: e3 54     LD   R5, @R4
7bc: 04 e5 15  ADD  15h, R5
7bf: 4e        INC  R4
7c0: a6 e4 0a  CP   R4, #0Ah
7c3: eb f5     JR   NZ, 07BAh
7c5: 4c 1f     LD   R4, #1Fh
7c7: e3 54     LD   R5, @R4
7c9: 04 e5 15  ADD  15h, R5
7cc: 4e        INC  R4
7cd: a6 e4 43  CP   R4, #43h
7d0: eb f5     JR   NZ, 07C7h
7d2: 31 10     SRP  #10h
7d4: af        RET  
7d5: ff        NOP  
7d6: ff        NOP  
7d7: ff        NOP  
7d8: ff        NOP  
7d9: ff        NOP  
7da: ff        NOP  
7db: ff        NOP  
7dc: ff        NOP  
7dd: ff        NOP  
7de: ff        NOP  
7df: ff        NOP  
7e0: ff        NOP  
7e1: ff        NOP  
7e2: ff        NOP  
7e3: ff        NOP  
7e4: ff        NOP  
7e5: ff        NOP  
7e6: ff        NOP  
7e7: ff        NOP  
7e8: ff        NOP  
7e9: ff        NOP  
7ea: ff        NOP  
7eb: ff        NOP  
7ec: ff        NOP  
7ed: ff        NOP  
7ee: ff        NOP  
7ef: ff        NOP  
7f0: ff        NOP  
7f1: ff        NOP  
7f2: ff        NOP  
7f3: ff        NOP  
7f4: ff        NOP  
7f5: ff        NOP  
7f6: ff        NOP  
7f7: ff        NOP  
7f8: ff        NOP  
7f9: ff        NOP  
7fa: ff        NOP  
7fb: ff        NOP  
7fc: ff        NOP  
7fd: ff        NOP  
7fe: ff        NOP  
7ff: ff        NOP  
800: 33 35     SBC  R3, @R5
802: 36 3d 3c  SBC  3Dh, #3Ch
805: 3b 3a     JR   ULE, 0841h
807: 31 64     SRP  #64h
809: 83 0a     LDEI @R0, @RR10
80b: 46 44 4b  OR   44h, #4Bh
80e: 49 13     LD   13h, R4
810: 52 54     AND  R5, R4
812: 4e        INC  R4
813: 45 4d 4c  OR   4Ch, @4Dh
816: 5d 4a 03  JP   MI, 4A03h
819: 66 01 09  TCM  P1, #09h
81c: 6a 5d     DJNZ R6, 087Bh
81e: 5a 29     DJNZ R5, 0849h
820: 0b 5b     JR   F, 087Dh
822: 55 3e 43  AND  43h, @3Eh
825: 42 41     OR   R4, R1
827: 51 04     POP  @04h
829: 6b 71     JR   Z, 089Ch
82b: 78 6c     LD   R7, 6Ch
82d: 69 77     LD   77h, R6
82f: 72 70     TM   R7, R0
831: 73 70     TM   R7, @R0
833: 07 75 72  ADD  @75h, #72h
836: 4a 74     DJNZ R4, 08ACh
838: ff        NOP  
839: 12 ff     ADC  R15, R15
83b: ff        NOP  
83c: ff        NOP  
83d: ff        NOP  
83e: 59 ff     LD   SPL, R5
840: 11 ff     RLC  @FFh
842: ff        NOP  
843: 7c 7e     LD   R7, #7Eh
845: ff        NOP  
846: ff        NOP  
847: 11 75     RLC  @75h
849: 79 6c     LD   6Ch, R7
84b: 69 6d     LD   6Dh, R6
84d: 5a 77     DJNZ R5, 08C6h
84f: 6b 71     JR   Z, 08C2h
851: 74 7d 7a  TM   7Ah, 7Dh
854: 7d 7a 7c  JP   C, 7A7Ch
857: 7b ff     JR   C, 0858h
859: ff        NOP  
85a: 14 ff ff  ADC  SPL, SPL
85d: ff        NOP  
85e: 14 ff 34  ADC  34h, SPL
861: 2c 2e     LD   R2, #2Eh
863: 25 2d 2b  SUB  2Bh, @2Dh
866: 2a 32     DJNZ R2, 089Ah
868: 0c 04     LD   R0, #04h
86a: 06 26 24  ADD  26h, #24h
86d: 23 21     SUB  R2, @R1
86f: ff        NOP  
870: 61 58     COM  @58h
872: 05 1e 1d  ADD  1Dh, @1Eh
875: 1b 22     JR   LT, 0899h
877: ff        NOP  
878: 76 0d 0e  TM   0Dh, #0Eh
87b: 16 15 1c  ADC  15h, #1Ch
87e: 1a 67     DJNZ R1, 08E7h
880: 33 84     SBC  R8, @R4
882: ff        NOP  
883: e0 12     RR   12h
885: e0 7c     RR   7Ch
887: 00 e0     DEC  R0
889: f0 7c     SWAP 7Ch
88b: 00 e1     DEC  R1
88d: 14 77 e1  ADC  R1, 77h
890: f0 14     SWAP 14h
892: f0 77     SWAP 77h
894: 00 e0     DEC  R0
896: 7e        INC  R7
897: e0 f0     RR   SIO
899: 7e        INC  R7
89a: 00 e0     DEC  R0
89c: f0 12     SWAP 12h
89e: 00 e0     DEC  R0
8a0: f0 59     SWAP 59h
8a2: 00 e0     DEC  R0
8a4: 59 00     LD   P0, R5
8a6: e0 12     RR   12h
8a8: 00 e0     DEC  R0
8aa: 2a e0     DJNZ R2, 088Ch
8ac: 37 00 e0  SBC  @00h, #E0h
8af: b7 00 00  XOR  @00h, #00h
8b2: e1 1d     RR   @1Dh
8b4: 45 e1 9d  OR   9Dh, @R1
8b7: c5        Illegal
8b8: 00 00     DEC  P0
8ba: 00 e0     DEC  R0
8bc: 46 e0 c6  OR   R0, #C6h
8bf: 00 00     DEC  P0
8c1: e0 aa     RR   AAh
8c3: 00 00     DEC  P0
8c5: e0 b6     RR   B6h
8c7: 00 00     DEC  P0
8c9: e0 36     RR   36h
8cb: 00 e0     DEC  R0
8cd: 2a 00     DJNZ R2, 08CFh
8cf: d6 0c cb  CALL 0CCBh
8d2: 60 ea     COM  R10
8d4: 6b 11     JR   Z, 08E7h
8d6: d6 08 dc  CALL 08DCh
8d9: 06 13 11  ADD  13h, #11h
8dc: 4c 20     LD   R4, #20h
8de: 04 13 e4  ADD  R4, 13h
8e1: e3 24     LD   R2, @R4
8e3: 52 2a     AND  R2, R10
8e5: f3 42     LD   @R4, R2
8e7: af        RET  
8e8: d6 0c cb  CALL 0CCBh
8eb: a6 ea ff  CP   R10, #FFh
8ee: 6b 21     JR   Z, 0911h
8f0: d6 09 06  CALL 0906h
8f3: 60 ea     COM  R10
8f5: 8d 08 d9  JP   08D9h
8f8: d6 0c cb  CALL 0CCBh
8fb: a6 ea ff  CP   R10, #FFh
8fe: 6b 11     JR   Z, 0911h
900: d6 09 06  CALL 0906h
903: 06 13 11  ADD  13h, #11h
906: 4c 20     LD   R4, #20h
908: 04 13 e4  ADD  R4, 13h
90b: e3 24     LD   R2, @R4
90d: 42 2a     OR   R2, R10
90f: f3 42     LD   @R4, R2
911: af        RET  
912: 4c 05     LD   R4, #05h
914: 4a fe     DJNZ R4, 0914h
916: 46 02 80  OR   P2, #80h
919: 4c 03     LD   R4, #03h
91b: 4a fe     DJNZ R4, 091Bh
91d: 76 e2 01  TM   R2, #01h
920: 6b 08     JR   Z, 092Ah
922: 46 02 40  OR   P2, #40h
925: ff        NOP  
926: ff        NOP  
927: ff        NOP  
928: 8b 09     JR   0933h
92a: 76 02 80  TM   P2, #80h
92d: 6b 16     JR   Z, 0945h
92f: ff        NOP  
930: 56 02 bf  AND  P2, #BFh
933: 4c 04     LD   R4, #04h
935: 4a fe     DJNZ R4, 0935h
937: 76 02 80  TM   P2, #80h
93a: 6b 09     JR   Z, 0945h
93c: 56 02 7f  AND  P2, #7Fh
93f: 4c 02     LD   R4, #02h
941: 4a fe     DJNZ R4, 0941h
943: cf        RCF  
944: af        RET  
945: df        SCF  
946: af        RET  
947: 23 15     SUB  R1, @R5
949: 07 08 16  ADD  @08h, #16h
94c: 24 32 31  SUB  31h, 32h
94f: 79 41     LD   41h, R7
951: 42 0a     OR   R0, R10
953: 18 26     LD   R1, 26h
955: 34 70 28  SBC  28h, 70h
958: 1a 0c     DJNZ R1, 0966h
95a: 0b 19     JR   F, 0975h
95c: 27 2b 35  SUB  @2Bh, #35h
95f: 3f        Illegal
960: 0e        INC  R0
961: 43 44     OR   R4, @R4
963: 7d 2b 1c  JP   C, 2B1Ch
966: 39 40     LD   40h, R3
968: 1b 0d     JR   LT, 0977h
96a: 09 17     LD   17h, R0
96c: 25 33 73  SUB  73h, @33h
96f: 3d 4b 53  JP   ULE, 4B53h
972: 57 47 4f  AND  @47h, #4Fh
975: 45 50 52  OR   52h, @50h
978: 4c 52     LD   R4, #52h
97a: 58 48     LD   R5, 48h
97c: 50 35     POP  35h
97e: 4d ff 2a  JP   OV, FF2Ah
981: ff        NOP  
982: ff        NOP  
983: ff        NOP  
984: ff        NOP  
985: 36 ff 38  SBC  SPL, #38h
988: ff        NOP  
989: ff        NOP  
98a: 37 46 ff  SBC  @46h, #FFh
98d: ff        NOP  
98e: 38 48     LD   R3, 48h
990: 4e        INC  R4
991: 47 4f 7e  OR   @4Fh, #7Eh
994: 1c 45     LD   R1, #45h
996: 4b 53     JR   OV, 09EBh
998: 4d 49 51  JP   OV, 4951h
99b: 49 51     LD   51h, R4
99d: 37 4a ff  SBC  @4Ah, #FFh
9a0: ff        NOP  
9a1: 1d ff ff  JP   LT, FFFFh
9a4: ff        NOP  
9a5: 1d ff 22  JP   LT, FF22h
9a8: 14 06 05  ADC  05h, 06h
9ab: 13 21     ADC  R2, @R1
9ad: 2f        Illegal
9ae: 30 3e     JP   @3Eh
9b0: 3d 3c 04  JP   ULE, 3C04h
9b3: 12 20     ADC  R2, R0
9b5: 2e        INC  R2
9b6: ff        NOP  
9b7: 56 3a 3b  AND  3Ah, #3Bh
9ba: 03 11     ADD  R1, @R1
9bc: 1f        Illegal
9bd: 2d ff 01  JP   LE, FF01h
9c0: 0f        Illegal
9c1: 29 02     LD   P2, R2
9c3: 10 1e     RLC  1Eh
9c5: 2c 7b     LD   R2, #7Bh
9c7: 23 54     SUB  R5, @R4
9c9: ff        NOP  
9ca: e6 f6 70  LD   P2M, #70h
9cd: 5f        Illegal
9ce: e6 02 ff  LD   P2, #FFh
9d1: 76 02 80  TM   P2, #80h
9d4: 6b f7     JR   Z, 09CDh
9d6: 4c 14     LD   R4, #14h
9d8: 4a fe     DJNZ R4, 09D8h
9da: 76 02 40  TM   P2, #40h
9dd: eb 78     JR   NZ, 0A57h
9df: 4c 08     LD   R4, #08h
9e1: d6 0c 39  CALL 0C39h
9e4: 76 02 40  TM   P2, #40h
9e7: eb 03     JR   NZ, 09ECh
9e9: cf        RCF  
9ea: 8b 01     JR   09EDh
9ec: df        SCF  
9ed: c0 e2     RRC  R2
9ef: 76 02 80  TM   P2, #80h
9f2: 6b 5e     JR   Z, 0A52h
9f4: 4a eb     DJNZ R4, 09E1h
9f6: b0 e6     CLR  R6
9f8: d6 0c 39  CALL 0C39h
9fb: 76 02 40  TM   P2, #40h
9fe: 6b 02     JR   Z, 0A02h
a00: 60 e6     COM  R6
a02: bc 03     LD   R11, #03h
a04: ba fe     DJNZ R11, 0A04h
a06: b0 ea     CLR  R10
a08: d6 0c 39  CALL 0C39h
a0b: 76 02 40  TM   P2, #40h
a0e: eb 02     JR   NZ, 0A12h
a10: 60 ea     COM  R10
a12: e6 f6 30  LD   P2M, #30h
a15: bc 02     LD   R11, #02h
a17: ba fe     DJNZ R11, 0A17h
a19: 56 02 bf  AND  P2, #BFh
a1c: d6 0c 39  CALL 0C39h
a1f: 46 02 40  OR   P2, #40h
a22: 56 ea ff  AND  R10, #FFh
a25: eb db     JR   NZ, 0A02h
a27: a8 e2     LD   R10, R2
a29: b0 e5     CLR  R5
a2b: 4c 08     LD   R4, #08h
a2d: 76 ea 01  TM   R10, #01h
a30: eb 02     JR   NZ, 0A34h
a32: 60 e5     COM  R5
a34: e0 ea     RR   R10
a36: 4a f5     DJNZ R4, 0A2Dh
a38: 56 e5 ff  AND  R5, #FFh
a3b: eb 08     JR   NZ, 0A45h
a3d: 56 e6 ff  AND  R6, #FFh
a40: eb 08     JR   NZ, 0A4Ah
a42: 8d 0a 52  JP   0A52h
a45: 56 e6 ff  AND  R6, #FFh
a48: eb 08     JR   NZ, 0A52h
a4a: cf        RCF  
a4b: e6 02 ff  LD   P2, #FFh
a4e: e6 f6 30  LD   P2M, #30h
a51: af        RET  
a52: b0 e4     CLR  R4
a54: df        SCF  
a55: 8b f4     JR   0A4Bh
a57: 4c ff     LD   R4, #FFh
a59: 8b f9     JR   0A54h
a5b: 28 ea     LD   R2, R10
a5d: 76 0e ff  TM   0Eh, #FFh
a60: 6b 5c     JR   Z, 0ABEh
a62: 76 0e 01  TM   0Eh, #01h
a65: eb 5a     JR   NZ, 0AC1h
a67: 76 0e 02  TM   0Eh, #02h
a6a: ed 0a f3  JP   NZ, 0AF3h
a6d: 76 0e 04  TM   0Eh, #04h
a70: ed 0b 01  JP   NZ, 0B01h
a73: 76 0e 08  TM   0Eh, #08h
a76: ed 0b 06  JP   NZ, 0B06h
a79: 76 0e 10  TM   0Eh, #10h
a7c: ed 0b 0b  JP   NZ, 0B0Bh
a7f: 76 0e 20  TM   0Eh, #20h
a82: 6b 3a     JR   Z, 0ABEh
a84: 76 e2 f8  TM   R2, #F8h
a87: eb 42     JR   NZ, 0ACBh
a89: 76 e2 02  TM   R2, #02h
a8c: eb 08     JR   NZ, 0A96h
a8e: 56 18 fd  AND  18h, #FDh
a91: 46 03 10  OR   P3, #10h
a94: 8b 06     JR   0A9Ch
a96: 46 18 02  OR   18h, #02h
a99: 56 03 ef  AND  P3, #EFh
a9c: 76 e2 01  TM   R2, #01h
a9f: eb 05     JR   NZ, 0AA6h
aa1: 46 03 80  OR   P3, #80h
aa4: 8b 03     JR   0AA9h
aa6: 56 03 7f  AND  P3, #7Fh
aa9: 76 e2 04  TM   R2, #04h
aac: eb 05     JR   NZ, 0AB3h
aae: 46 03 20  OR   P3, #20h
ab1: 8b 03     JR   0AB6h
ab3: 56 03 df  AND  P3, #DFh
ab6: d6 0c 22  CALL 0C22h
ab9: 56 0e df  AND  0Eh, #DFh
abc: 8b 40     JR   0AFEh
abe: 8d 0b 56  JP   0B56h
ac1: 76 e2 ff  TM   R2, #FFh
ac4: 6b 0d     JR   Z, 0AD3h
ac6: 76 e2 fc  TM   R2, #FCh
ac9: 6b 12     JR   Z, 0ADDh
acb: 2c fe     LD   R2, #FEh
acd: d6 0c 24  CALL 0C24h
ad0: 8d 0b 11  JP   0B11h
ad3: d6 0c 22  CALL 0C22h
ad6: 28 09     LD   R2, 09h
ad8: d6 0c 24  CALL 0C24h
adb: 8b 21     JR   0AFEh
add: b0 08     CLR  08h
adf: 29 09     LD   09h, R2
ae1: d6 0c 22  CALL 0C22h
ae4: a6 09 01  CP   09h, #01h
ae7: eb 03     JR   NZ, 0AECh
ae9: e6 08 26  LD   08h, #26h
aec: d6 0d 2f  CALL 0D2Fh
aef: b0 0b     CLR  0Bh
af1: 8b 0b     JR   0AFEh
af3: 76 e2 80  TM   R2, #80h
af6: eb d3     JR   NZ, 0ACBh
af8: d6 07 3f  CALL 073Fh
afb: d6 0c 22  CALL 0C22h
afe: 8d 0c 0f  JP   0C0Fh
b01: d6 08 f8  CALL 08F8h
b04: 8b 08     JR   0B0Eh
b06: d6 08 cf  CALL 08CFh
b09: 8b 03     JR   0B0Eh
b0b: d6 08 e8  CALL 08E8h
b0e: 8d 0b 11  JP   0B11h
b11: 5f        Illegal
b12: e6 0d 55  LD   0Dh, #55h
b15: e6 68 20  LD   68h, #20h
b18: 8f        DI   
b19: d6 09 ca  CALL 09CAh
b1c: 7d 0b 56  JP   C, 0B56h
b1f: 9f        EI   
b20: cf        RCF  
b21: 06 e2 13  ADD  R2, #13h
b24: fd 0a 5b  JP   NC, 0A5Bh
b27: 0c 0b     LD   R0, #0Bh
b29: 1c 33     LD   R1, #33h
b2b: 02 12     ADD  R1, R2
b2d: c2 20     LDC  R2, @RR0
b2f: 18 e2     LD   R1, R2
b31: 30 e0     JP   @RR0
b33: 46 4e 56  OR   4Eh, #56h
b36: 65 5d 6a  TCM  6Ah, @5Dh
b39: 7d 82 8b  JP   C, 828Bh
b3c: 97        Illegal
b3d: a0 a9     INCW A9h
b3f: b6 c9 d2  XOR  C9h, #D2h
b42: d7 dc e7  LD   R12, E7h(R13)
b45: ee        INC  R14
b46: e6 0e 20  LD   0Eh, #20h
b49: d6 0c 22  CALL 0C22h
b4c: 8b c3     JR   0B11h
b4e: 2c ee     LD   R2, #EEh
b50: d6 0c 24  CALL 0C24h
b53: 8d 0c 0f  JP   0C0Fh
b56: 9f        EI   
b57: a6 e4 ff  CP   R4, #FFh
b5a: 6d 0c 11  JP   Z, 0C11h
b5d: 2c fe     LD   R2, #FEh
b5f: d6 0c 24  CALL 0C24h
b62: 8d 0c 11  JP   0C11h
b65: e6 0e 01  LD   0Eh, #01h
b68: 8b df     JR   0B49h
b6a: d6 0c 22  CALL 0C22h
b6d: 2c ab     LD   R2, #ABh
b6f: d6 0c 24  CALL 0C24h
b72: 2c 83     LD   R2, #83h
b74: d6 0c 24  CALL 0C24h
b77: 46 1f 40  OR   1Fh, #40h
b7a: 8d 00 7a  JP   007Ah
b7d: e6 0e 02  LD   0Eh, #02h
b80: 8b c7     JR   0B49h
b82: d6 0d 24  CALL 0D24h
b85: 46 1f 40  OR   1Fh, #40h
b88: 8d 00 7a  JP   007Ah
b8b: d6 06 67  CALL 0667h
b8e: d6 0d 24  CALL 0D24h
b91: 56 1f bf  AND  1Fh, #BFh
b94: 8d 0b 11  JP   0B11h
b97: d6 0d 24  CALL 0D24h
b9a: d6 06 67  CALL 0667h
b9d: 8d 0c 11  JP   0C11h
ba0: 4c 31     LD   R4, #31h
ba2: 5c ff     LD   R5, #FFh
ba4: d6 0e 5b  CALL 0E5Bh
ba7: 8b 14     JR   0BBDh
ba9: 4c 31     LD   R4, #31h
bab: b0 e5     CLR  R5
bad: d6 0e 5b  CALL 0E5Bh
bb0: 4c 20     LD   R4, #20h
bb2: b0 e5     CLR  R5
bb4: 8b 0b     JR   0BC1h
bb6: 4c 31     LD   R4, #31h
bb8: b0 e5     CLR  R5
bba: d6 0e 5b  CALL 0E5Bh
bbd: 4c 20     LD   R4, #20h
bbf: 5c ff     LD   R5, #FFh
bc1: d6 0e 5b  CALL 0E5Bh
bc4: d6 0c 22  CALL 0C22h
bc7: 8b 46     JR   0C0Fh
bc9: 4c 31     LD   R4, #31h
bcb: 5c ff     LD   R5, #FFh
bcd: d6 0e 5b  CALL 0E5Bh
bd0: 8b de     JR   0BB0h
bd2: e6 0e 04  LD   0Eh, #04h
bd5: 8b 08     JR   0BDFh
bd7: e6 0e 08  LD   0Eh, #08h
bda: 8b 03     JR   0BDFh
bdc: e6 0e 10  LD   0Eh, #10h
bdf: d6 0d 2f  CALL 0D2Fh
be2: d6 0c 22  CALL 0C22h
be5: 8b aa     JR   0B91h
be7: 28 0f     LD   R2, 0Fh
be9: d6 0c 24  CALL 0C24h
bec: 8b 23     JR   0C11h
bee: d6 0c 22  CALL 0C22h
bf1: d6 0d 2f  CALL 0D2Fh
bf4: 8f        DI   
bf5: 4c 1e     LD   R4, #1Eh
bf7: 5f        Illegal
bf8: 76 02 80  TM   P2, #80h
bfb: 6b f8     JR   Z, 0BF5h
bfd: 76 02 40  TM   P2, #40h
c00: 6b f3     JR   Z, 0BF5h
c02: 4a f3     DJNZ R4, 0BF7h
c04: 76 02 40  TM   P2, #40h
c07: 6d 0b 11  JP   Z, 0B11h
c0a: b0 08     CLR  08h
c0c: 8d 00 0d  JP   000Dh
c0f: b0 0e     CLR  0Eh
c11: 76 0e ff  TM   0Eh, #FFh
c14: ed 0b 11  JP   NZ, 0B11h
c17: 76 1f 40  TM   1Fh, #40h
c1a: eb 03     JR   NZ, 0C1Fh
c1c: 8d 0b 11  JP   0B11h
c1f: 8d 00 7a  JP   007Ah
c22: 2c fa     LD   R2, #FAh
c24: 68 e2     LD   R6, R2
c26: 8f        DI   
c27: 5f        Illegal
c28: d6 0e d6  CALL 0ED6h
c2b: 7b 01     JR   C, 0C2Eh
c2d: af        RET  
c2e: 9f        EI   
c2f: 5c 19     LD   R5, #19h
c31: 5a fe     DJNZ R5, 0C31h
c33: 76 02 40  TM   P2, #40h
c36: eb ee     JR   NZ, 0C26h
c38: af        RET  
c39: 56 02 7f  AND  P2, #7Fh
c3c: bc 0e     LD   R11, #0Eh
c3e: ba fe     DJNZ R11, 0C3Eh
c40: 46 02 80  OR   P2, #80h
c43: bc 05     LD   R11, #05h
c45: ba fe     DJNZ R11, 0C45h
c47: af        RET  
c48: 33 35     SBC  R3, @R5
c4a: 36 3d 3c  SBC  3Dh, #3Ch
c4d: 3b 3a     JR   ULE, 0C89h
c4f: 31 86     SRP  #86h
c51: 37 3f 46  SBC  @3Fh, #46h
c54: 44 4b 49  OR   49h, 4Bh
c57: 87        Illegal
c58: 52 54     AND  R5, R4
c5a: 4e        INC  R4
c5b: 45 4d 4c  OR   4Ch, @4Dh
c5e: 53 4a     AND  R4, @R10
c60: 27 66 47  SUB  @66h, #47h
c63: 4f        Illegal
c64: 5d 5c 5a  JP   MI, 5C5Ah
c67: 29 2f     LD   2Fh, R2
c69: 5b 55     JR   MI, 0CC0h
c6b: 3e        INC  R3
c6c: 43 42     OR   R4, @R2
c6e: 41 51     DA   @51h
c70: 0c 6b     LD   R0, #6Bh
c72: 64 56 6c  TCM  6Ch, 56h
c75: 69 76     LD   76h, R6
c77: 60 70     COM  70h
c79: 73 67     TM   R6, @R7
c7b: 5e        INC  R5
c7c: 75 72 77  TM   77h, @72h
c7f: 6a ff     DJNZ R6, 0C80h
c81: 12 ff     ADC  R15, R15
c83: ff        NOP  
c84: ff        NOP  
c85: ff        NOP  
c86: 59 ff     LD   SPL, R5
c88: 19 ff     LD   SPL, R1
c8a: ff        NOP  
c8b: 57 5f ff  AND  @5Fh, #FFh
c8e: ff        NOP  
c8f: 39 63     LD   63h, R3
c91: 7c 6e     LD   R7, #6Eh
c93: 65 7b 79  TCM  79h, @7Bh
c96: 62 61     TCM  R6, R1
c98: 71 74     PUSH @74h
c9a: 6f        Illegal
c9b: 6d 7d 7a  JP   Z, 7D7Ah
c9e: 7e        INC  R7
c9f: 84        Illegal
ca0: ff        NOP  
ca1: ff        NOP  
ca2: 11 ff     RLC  @FFh
ca4: ff        NOP  
ca5: ff        NOP  
ca6: 58 ff     LD   R5, SPL
ca8: 34 2c 2e  SBC  2Eh, 2Ch
cab: 25 2d 2b  SUB  2Bh, @2Dh
cae: 2a 32     DJNZ R2, 0CE2h
cb0: 1f        Illegal
cb1: 17 0f 26  ADC  @0Fh, #26h
cb4: 24 23 21  SUB  21h, 23h
cb7: ff        NOP  
cb8: 13 14     ADC  R1, @R4
cba: 07 1e 1d  ADD  @1Eh, #1Dh
cbd: 1b 22     JR   LT, 0CE1h
cbf: ff        NOP  
cc0: 08 0d     LD   R0, 0Dh
cc2: 0e        INC  R0
cc3: 16 15 1c  ADC  15h, #1Ch
cc6: 1a 85     DJNZ R1, 0C4Dh
cc8: 33 ff     SBC  R15, @R15
cca: ff        NOP  
ccb: a6 e2 84  CP   R2, #84h
cce: 6b 14     JR   Z, 0CE4h
cd0: a6 e2 85  CP   R2, #85h
cd3: 6b 0f     JR   Z, 0CE4h
cd5: a6 e2 86  CP   R2, #86h
cd8: 6b 0a     JR   Z, 0CE4h
cda: a6 e2 87  CP   R2, #87h
cdd: 6b 05     JR   Z, 0CE4h
cdf: 76 e2 80  TM   R2, #80h
ce2: eb 38     JR   NZ, 0D1Ch
ce4: 1c 4b     LD   R1, #4Bh
ce6: 0c 0d     LD   R0, #0Dh
ce8: 02 12     ADD  R1, R2
cea: c2 20     LDC  R2, @RR0
cec: 68 e2     LD   R6, R2
cee: a6 e6 ff  CP   R6, #FFh
cf1: eb 04     JR   NZ, 0CF7h
cf3: 2c fa     LD   R2, #FAh
cf5: 8b 27     JR   0D1Eh
cf7: 2c fa     LD   R2, #FAh
cf9: 70 e6     PUSH R6
cfb: d6 0c 24  CALL 0C24h
cfe: 50 e6     POP  R6
d00: 69 13     LD   13h, R6
d02: e0 13     RR   13h
d04: e0 13     RR   13h
d06: e0 13     RR   13h
d08: 56 13 1f  AND  13h, #1Fh
d0b: a8 e6     LD   R10, R6
d0d: 56 ea 07  AND  R10, #07h
d10: 4c 01     LD   R4, #01h
d12: ae        INC  R10
d13: aa 03     DJNZ R10, 0D18h
d15: a8 e4     LD   R10, R4
d17: af        RET  
d18: 90 e4     RL   R4
d1a: 8b f7     JR   0D13h
d1c: 2c fe     LD   R2, #FEh
d1e: d6 0c 24  CALL 0C24h
d21: ac ff     LD   R10, #FFh
d23: af        RET  
d24: d6 0d 2f  CALL 0D2Fh
d27: d6 0c 22  CALL 0C22h
d2a: b0 0b     CLR  0Bh
d2c: b0 0e     CLR  0Eh
d2e: af        RET  
d2f: 4c 44     LD   R4, #44h
d31: b1 e4     CLR  @R4
d33: 4e        INC  R4
d34: a6 e4 55  CP   R4, #55h
d37: eb f8     JR   NZ, 0D31h
d39: e6 0a 44  LD   0Ah, #44h
d3c: af        RET  
d3d: 4c 09     LD   R4, #09h
d3f: 5c 3e     LD   R5, #3Eh
d41: 6c c8     LD   R6, #C8h
d43: 5f        Illegal
d44: 6a fe     DJNZ R6, 0D44h
d46: 5a f9     DJNZ R5, 0D41h
d48: 4a f5     DJNZ R4, 0D3Fh
d4a: af        RET  
d4b: ff        NOP  
d4c: ff        NOP  
d4d: ff        NOP  
d4e: ff        NOP  
d4f: ff        NOP  
d50: ff        NOP  
d51: ff        NOP  
d52: 72 78     TM   R7, R8
d54: ff        NOP  
d55: ff        NOP  
d56: ff        NOP  
d57: 28 79     LD   R2, 79h
d59: 7a 6a     DJNZ R7, 0DC5h
d5b: ff        NOP  
d5c: 5a 39     DJNZ R5, 0D97h
d5e: 70 71     PUSH 71h
d60: 7c 7b     LD   R7, #7Bh
d62: 69 ff     LD   SPL, R6
d64: 40 7e     DA   7Eh
d66: 75 7d 74  TM   74h, @7Dh
d69: 73 68     TM   R6, @R8
d6b: ff        NOP  
d6c: 6e        INC  R6
d6d: 76 6d 6c  TM   6Dh, #6Ch
d70: 63 6b     TCM  R6, @R11
d72: 18 ff     LD   R1, SPL
d74: 1f        Illegal
d75: 66 65 61  TCM  65h, #61h
d78: 64 62 20  TCM  20h, 62h
d7b: ff        NOP  
d7c: 07 67 80  ADD  @67h, #80h
d7f: 60 01     COM  P1
d81: 02 09     ADD  R0, R9
d83: ff        NOP  
d84: 47 06 05  OR   @06h, #05h
d87: 04 03 23  ADD  23h, P3
d8a: 0a ff     DJNZ R0, 0D8Bh
d8c: 26 25 24  SUB  25h, #24h
d8f: 0c 13     LD   R0, #13h
d91: 0b 1a     JR   F, 0DADh
d93: ff        NOP  
d94: 0e        INC  R0
d95: 17 0d 15  ADC  @0Dh, #15h
d98: 14 12 1b  ADC  1Bh, 12h
d9b: ff        NOP  
d9c: 27 10 16  SUB  @10h, #16h
d9f: 11 22     RLC  @22h
da1: 2b 43     JR   LE, 0DE6h
da3: 5e        INC  R5
da4: 3e        INC  R3
da5: 1e        INC  R1
da6: 21 1d     INC  @1Dh
da8: 1c 33     LD   R1, #33h
daa: 44 2f 4f  OR   4Fh, 2Fh
dad: 4e        INC  R4
dae: 48 2a     LD   R4, 2Ah
db0: 4b 19     JR   OV, 0DCBh
db2: 32 ff     SBC  R15, R15
db4: 2d 37 29  JP   LE, 3729h
db7: 2c 53     LD   R2, #53h
db9: 4a 52     DJNZ R4, 0E0Dh
dbb: 30 50     JP   @50h
dbd: 35 31 51  SBC  51h, @31h
dc0: 34 2e 36  SBC  36h, 2Eh
dc3: ff        NOP  
dc4: 4d 55 4c  JP   OV, 554Ch
dc7: 49 54     LD   54h, R4
dc9: 56 27 ff  AND  27h, #FFh
dcc: ff        NOP  
dcd: ff        NOP  
dce: ff        NOP  
dcf: 57 7f 08  AND  @7Fh, #08h
dd2: 0f        Illegal
dd3: 28 e6     LD   R2, R6
dd5: b0 ea     CLR  R10
dd7: bc 08     LD   R11, #08h
dd9: 76 e2 01  TM   R2, #01h
ddc: eb 01     JR   NZ, 0DDFh
dde: ae        INC  R10
ddf: e0 e2     RR   R2
de1: ba f6     DJNZ R11, 0DD9h
de3: 76 ea 01  TM   R10, #01h
de6: eb 03     JR   NZ, 0DEBh
de8: ac 03     LD   R10, #03h
dea: af        RET  
deb: ac 02     LD   R10, #02h
ded: af        RET  
dee: 28 ec     LD   R2, R12
df0: d6 0e 26  CALL 0E26h
df3: 76 05 02  TM   05h, #02h
df6: eb 2d     JR   NZ, 0E25h
df8: 2c f0     LD   R2, #F0h
dfa: d6 07 8a  CALL 078Ah
dfd: 8b 11     JR   0E10h
dff: a6 0b 82  CP   0Bh, #82h
e02: 6b 0a     JR   Z, 0E0Eh
e04: 28 0b     LD   R2, 0Bh
e06: d6 0e 26  CALL 0E26h
e09: 76 05 01  TM   05h, #01h
e0c: 6b 17     JR   Z, 0E25h
e0e: c8 0b     LD   R12, 0Bh
e10: 0c 0c     LD   R0, #0Ch
e12: 1c 48     LD   R1, #48h
e14: 02 1c     ADD  R1, R12
e16: c2 20     LDC  R2, @RR0
e18: a6 e2 ff  CP   R2, #FFh
e1b: eb 05     JR   NZ, 0E22h
e1d: b0 0b     CLR  0Bh
e1f: e4 06 0c  LD   0Ch, 06h
e22: d6 07 8a  CALL 078Ah
e25: af        RET  
e26: b0 05     CLR  05h
e28: a8 e2     LD   R10, R2
e2a: 56 ea 07  AND  R10, #07h
e2d: b8 ea     LD   R11, R10
e2f: 58 e2     LD   R5, R2
e31: e0 e5     RR   R5
e33: e0 e5     RR   R5
e35: e0 e5     RR   R5
e37: 56 e5 1f  AND  R5, #1Fh
e3a: 06 e5 20  ADD  R5, #20h
e3d: e3 25     LD   R2, @R5
e3f: ae        INC  R10
e40: cf        RCF  
e41: c0 e2     RRC  R2
e43: aa fc     DJNZ R10, 0E41h
e45: fb 03     JR   NC, 0E4Ah
e47: 46 05 02  OR   05h, #02h
e4a: 06 e5 11  ADD  R5, #11h
e4d: e3 25     LD   R2, @R5
e4f: be        INC  R11
e50: cf        RCF  
e51: c0 e2     RRC  R2
e53: ba fc     DJNZ R11, 0E51h
e55: fb 03     JR   NC, 0E5Ah
e57: 46 05 01  OR   05h, #01h
e5a: af        RET  
e5b: 6c 11     LD   R6, #11h
e5d: f3 45     LD   @R4, R5
e5f: 4e        INC  R4
e60: 6a fb     DJNZ R6, 0E5Dh
e62: d6 0d 2f  CALL 0D2Fh
e65: af        RET  
e66: a6 0b 00  CP   0Bh, #00h
e69: 6b 35     JR   Z, 0EA0h
e6b: a6 0c 00  CP   0Ch, #00h
e6e: eb 30     JR   NZ, 0EA0h
e70: e4 07 0c  LD   0Ch, 07h
e73: a6 44 00  CP   44h, #00h
e76: eb 21     JR   NZ, 0E99h
e78: a6 09 03  CP   09h, #03h
e7b: 6b 20     JR   Z, 0E9Dh
e7d: c8 0b     LD   R12, 0Bh
e7f: d6 02 25  CALL 0225h
e82: 76 ee 01  TM   R14, #01h
e85: eb 1a     JR   NZ, 0EA1h
e87: 76 ee 02  TM   R14, #02h
e8a: eb 0d     JR   NZ, 0E99h
e8c: 76 ee 04  TM   R14, #04h
e8f: eb 1c     JR   NZ, 0EADh
e91: 76 ee 18  TM   R14, #18h
e94: eb 17     JR   NZ, 0EADh
e96: d6 0e b6  CALL 0EB6h
e99: 56 18 7f  AND  18h, #7Fh
e9c: af        RET  
e9d: d6 0d ff  CALL 0DFFh
ea0: af        RET  
ea1: 76 18 08  TM   18h, #08h
ea4: 6b 07     JR   Z, 0EADh
ea6: cc 81     LD   R12, #81h
ea8: d6 0e b6  CALL 0EB6h
eab: 8b ec     JR   0E99h
ead: 2c e0     LD   R2, #E0h
eaf: d6 07 8a  CALL 078Ah
eb2: c8 0b     LD   R12, 0Bh
eb4: 8b e0     JR   0E96h
eb6: d6 0f d3  CALL 0FD3h
eb9: a6 08 00  CP   08h, #00h
ebc: 6b 0a     JR   Z, 0EC8h
ebe: d6 0f ca  CALL 0FCAh
ec1: a6 e2 ff  CP   R2, #FFh
ec4: 6b 07     JR   Z, 0ECDh
ec6: 8b 0a     JR   0ED2h
ec8: a6 e2 ff  CP   R2, #FFh
ecb: eb 05     JR   NZ, 0ED2h
ecd: b0 0b     CLR  0Bh
ecf: e4 06 0c  LD   0Ch, 06h
ed2: d6 07 8a  CALL 078Ah
ed5: af        RET  
ed6: 5f        Illegal
ed7: e6 02 ff  LD   P2, #FFh
eda: e6 0d 55  LD   0Dh, #55h
edd: e6 68 20  LD   68h, #20h
ee0: 76 02 80  TM   P2, #80h
ee3: 6b f1     JR   Z, 0ED6h
ee5: 5f        Illegal
ee6: e6 0d 55  LD   0Dh, #55h
ee9: e6 68 20  LD   68h, #20h
eec: a6 08 00  CP   08h, #00h
eef: eb 07     JR   NZ, 0EF8h
ef1: a6 e6 ff  CP   R6, #FFh
ef4: eb 02     JR   NZ, 0EF8h
ef6: b0 e6     CLR  R6
ef8: d6 0d d3  CALL 0DD3h
efb: bc 1e     LD   R11, #1Eh
efd: 76 02 80  TM   P2, #80h
f00: 6b 0c     JR   Z, 0F0Eh
f02: bc 0a     LD   R11, #0Ah
f04: ba fe     DJNZ R11, 0F04h
f06: 76 02 40  TM   P2, #40h
f09: eb 18     JR   NZ, 0F23h
f0b: 8f        DI   
f0c: df        SCF  
f0d: af        RET  
f0e: 5f        Illegal
f0f: 76 02 40  TM   P2, #40h
f12: 6b 02     JR   Z, 0F16h
f14: ba e7     DJNZ R11, 0EFDh
f16: 8b 08     JR   0F20h
f18: 5f        Illegal
f19: 76 02 40  TM   P2, #40h
f1c: 6b 02     JR   Z, 0F20h
f1e: ba 0c     DJNZ R11, 0F2Ch
f20: 8f        DI   
f21: df        SCF  
f22: af        RET  
f23: 5f        Illegal
f24: 76 03 04  TM   P3, #04h
f27: eb 1c     JR   NZ, 0F45h
f29: bc 1e     LD   R11, #1Eh
f2b: 8f        DI   
f2c: e6 02 ff  LD   P2, #FFh
f2f: ff        NOP  
f30: 76 02 80  TM   P2, #80h
f33: 6b e3     JR   Z, 0F18h
f35: 56 02 bf  AND  P2, #BFh
f38: bc 03     LD   R11, #03h
f3a: ba fe     DJNZ R11, 0F3Ah
f3c: 56 02 3f  AND  P2, #3Fh
f3f: bc 05     LD   R11, #05h
f41: ba fe     DJNZ R11, 0F41h
f43: 8b 28     JR   0F6Dh
f45: 8f        DI   
f46: e6 6a 0f  LD   6Ah, #0Fh
f49: e6 fb 90  LD   IMR, #90h
f4c: 46 f1 03  OR   TMR, #03h
f4f: 56 02 bf  AND  P2, #BFh
f52: ff        NOP  
f53: 46 02 80  OR   P2, #80h
f56: 76 02 80  TM   P2, #80h
f59: 6b fb     JR   Z, 0F56h
f5b: 56 02 3f  AND  P2, #3Fh
f5e: 8f        DI   
f5f: e6 fb 20  LD   IMR, #20h
f62: ff        NOP  
f63: 56 fb ef  AND  IMR, #EFh
f66: a6 6a 00  CP   6Ah, #00h
f69: 6b 34     JR   Z, 0F9Fh
f6b: b0 6a     CLR  6Ah
f6d: bc 08     LD   R11, #08h
f6f: 28 e6     LD   R2, R6
f71: d6 09 12  CALL 0912h
f74: 7b 29     JR   C, 0F9Fh
f76: e0 e2     RR   R2
f78: 00 eb     DEC  R11
f7a: eb f5     JR   NZ, 0F71h
f7c: 28 ea     LD   R2, R10
f7e: d6 09 12  CALL 0912h
f81: 7d 0f 9f  JP   C, 0F9Fh
f84: ff        NOP  
f85: ff        NOP  
f86: e0 e2     RR   R2
f88: d6 09 12  CALL 0912h
f8b: 7d 0f 9f  JP   C, 0F9Fh
f8e: bc 0a     LD   R11, #0Ah
f90: ba fe     DJNZ R11, 0F90h
f92: e6 02 ff  LD   P2, #FFh
f95: 9f        EI   
f96: a6 e6 fe  CP   R6, #FEh
f99: 6b 02     JR   Z, 0F9Dh
f9b: 69 0f     LD   0Fh, R6
f9d: cf        RCF  
f9e: af        RET  
f9f: e6 02 ff  LD   P2, #FFh
fa2: df        SCF  
fa3: af        RET  
fa4: 5f        Illegal
fa5: a6 6a 00  CP   6Ah, #00h
fa8: 6b 07     JR   Z, 0FB1h
faa: 00 6a     DEC  6Ah
fac: eb 03     JR   NZ, 0FB1h
fae: e6 02 ff  LD   P2, #FFh
fb1: bf        IRET 
fb2: a6 0c 00  CP   0Ch, #00h
fb5: 6b 03     JR   Z, 0FBAh
fb7: 00 0c     DEC  0Ch
fb9: bf        IRET 
fba: 00 68     DEC  68h
fbc: eb 0b     JR   NZ, 0FC9h
fbe: a6 0d 55  CP   0Dh, #55h
fc1: ed 00 0d  JP   NZ, 000Dh
fc4: b0 0d     CLR  0Dh
fc6: e6 68 16  LD   68h, #16h
fc9: bf        IRET 
fca: 1c 47     LD   R1, #47h
fcc: 0c 09     LD   R0, #09h
fce: 02 1c     ADD  R1, R12
fd0: c2 20     LDC  R2, @RR0
fd2: af        RET  
fd3: 1c 00     LD   R1, #00h
fd5: 0c 08     LD   R0, #08h
fd7: 02 1c     ADD  R1, R12
fd9: c2 20     LDC  R2, @RR0
fdb: af        RET  
fdc: df        SCF  
fdd: af        RET  
fde: b0 15     CLR  15h
fe0: 0c 0f     LD   R0, #0Fh
fe2: 1c ed     LD   R1, #EDh
fe4: c2 20     LDC  R2, @RR0
fe6: 04 e2 15  ADD  15h, R2
fe9: 5f        Illegal
fea: 80 e0     DECW R0
fec: eb f6     JR   NZ, 0FE4h
fee: a6 15 c4  CP   15h, #C4h
ff1: eb e9     JR   NZ, 0FDCh
ff3: cf        RCF  
ff4: af        RET  
ff5: ff        NOP  
ff6: ff        NOP  
ff7: ff        NOP  
ff8: ff        NOP  
ff9: ff        NOP  
ffa: ff        NOP  
ffb: ff        NOP  
ffc: ff        NOP  
ffd: ff        NOP  
ffe: ff        NOP  
fff: ff        NOP  
